:100000000C94F00C0C94180D0C94180D0C94421FC9
:100010000C94180D0C94180D0C94180D0C94180DCC
:100020000C94180D0C94180D0C94180D0C94180DBC
:100030000C94180D0C94180D0C94180D0C94180DAC
:100040000C94F81E0C94180D0C94180D0C94180DAB
:100050000C94180D0C9419200C94180D0C94180D78
:100060000C94180D0C94180D4465616374697661E5
:1000700074656400456E74657220546970204E6129
:100080006D6500FFE0FFD1AFFF32FFD0FFFEFFE064
:10009000FFD1AEFFD0FFFEFFE0FFD11000FFFEFF5B
:1000A000D0FFE0FFC1FFD1AED580A83FD300408D87
:1000B000142000A1C8DA1281CFD9F1DB402EA4A60A
:1000C000AFFFD0FFFE53656C656374205469700008
:1000D000506C6561736520776169742E2E2E004126
:1000E00044433A20200074656D703A2000536574D3
:1000F000206D6561737572656400537465703A2094
:100100000043616C6962726174696F6E0020560011
:100110005663633A20200020560056696E3A20004C
:10012000204300546D703A20004669726D77617209
:10013000653A200030303000303030005600204822
:100140004F4C4400204845415400574F524B5900F2
:10015000424F4F535400534C4545500020204F46CA
:1001600046004552524F5200000000002400270074
:100170002A0000000000250028002B0000000000DD
:1001800023002600290004040404040404040202D9
:100190000202020203030303030301020408102006
:1001A0004080010204081020010204081020000011
:1001B0000008000201000003040700000000000026
:1001C000000000574DFBF12A000000002A3A002BE6
:1001D000F82A001717452507140082000383800FB3
:1001E00083E01FC7E00FC7E007C7C003EF8001EF40
:1001F0000000FE00F8FE3EFFFFFEFFFFFEFFFFFED9
:10020000FE7CFE80FE0201EF0003EF8007EFC007D7
:10021000C7C00FC7E01F83F00783C00183002323FB
:10022000AF3B0C000001E000000001E00000000115
:10023000E000000001E000000001E000000001E03B
:1002400000000001E000000001E000000001E0000B
:10025000000001E000000001E000000001E00000FB
:100260000001E000000001E000000001E0000000EB
:1002700001E00000FFFFFFFFE0FFFFFFFFE0FFFFE7
:10028000FFFFE0FFFFFFFFE00001E000000001E0F2
:1002900000000001E000000001E000000001E000BB
:1002A000000001E000000001E000000001E00000AB
:1002B0000001E000000001E000000001E00000009B
:1002C00001E000000001E000000001E0000000018A
:1002D000E000000C0F1E1203F80FF00FF00FE01FEC
:1002E000E01FC01FC03F803F803F007F007E007E38
:1002F000007C00FC00FC000F081013020BFFFEFF47
:10030000FEFFFEFFFEFFFEFFFEFFFEFFFE080808E9
:10031000120600FFFFFFFFFFFFFFFF132E8A1903E6
:10032000FD0007E00007E00007C0000FC0000FC09D
:10033000000F80001F80001F80001F80001F000032
:100340003F00003F00003E00007E00007E00007C79
:100350000000FC0000FC0000FC0000F80001F800B8
:1003600001F80001F00003F00003F00003F00007C3
:10037000E00007E00007E00007C0000FC0000FC06A
:10038000000F80001F80001F80001F80003F0000C2
:100390003F00003F00003E00007E00007E00007C29
:1003A0000000FC0000FC0000FC00001D2CB021023D
:1003B000FF001FC00000FFF80003FFFC0007FFFF65
:1003C000000FFFFF800FFFFF801FF0FFC03FC03F07
:1003D000C03FC03FE03F801FE07F801FF07F001FD5
:1003E000F07F000FF07F000FF0FF000FF0FF000F15
:1003F000F8FF000FF8FF000FF8FF000FF8FF000FE5
:10040000F8FF000FF8FF000FF8FF000FF8FF000FD4
:10041000F8FF000FF8FF000FF8FF000FF8FF000FC4
:10042000F8FF000FF87F000FF07F000FF07F000F44
:10043000F07F001FF07F801FF03F801FE03FC03F34
:10044000E03FC03FC01FF0FFC00FFFFF800FFFFF66
:100450000007FFFF0003FFFE0000FFF800001FC0C1
:1004600000122A7E210600003FC0007FC000FFC0AE
:1004700003FFC00FFFC03FFFC0FFFFC0FFFFC0FF73
:10048000FFC0FF3FC0FE3FC0F83FC0E03FC0003F9D
:10049000C0003FC0003FC0003FC0003FC0003FC0A1
:1004A000003FC0003FC0003FC0003FC0003FC00051
:1004B0003FC0003FC0003FC0003FC0003FC0003F02
:1004C000C0003FC0003FC0003FC0003FC0003FC071
:1004D000003FC0003FC0003FC0003FC0003FC00021
:1004E0003FC0003FC01D2BAC210200000FF00000F8
:1004F0007FFE0001FFFF0003FFFF8007FFFFC00F2B
:10050000FFFFE01FF83FF01FF01FF01FE00FF03F6C
:10051000C007F83FC007F83FC007F8000007F80021
:100520000007F800000FF800000FF000001FF000B7
:10053000001FF000003FE000007FE00000FFC0006F
:1005400001FF800003FF800007FF00000FFE000096
:100550001FFC00003FF800007FF00000FFE00001FA
:10056000FF800003FF00000FFE00001FFC00003FA3
:10057000F000007FE00000FFC00000FFFFFFF8FF79
:10058000FFFFF8FFFFFFF8FFFFFFF8FFFFFFF8FF97
:10059000FFFFF8FFFFFFF81C2CB02103FF007FC016
:1005A0000003FFF80007FFFC001FFFFF003FFFFFF5
:1005B000003FFFFF807FE0FFC07FC07FC0FF803F24
:1005C000C0FF001FE0FF001FE0FF001FE000001F52
:1005D000E000001FE000001FE000003FC000007FBF
:1005E000C00003FF80007FFF00007FFC00007FF061
:1005F00000007FF800007FFE00007FFF800000FF0A
:10060000C000003FE000001FE000001FE000000FFE
:10061000F000000FF000000FF0FF000FF0FF000FE0
:10062000F0FF000FF0FF001FE0FF801FE07FC03FE2
:10063000E07FE0FFC03FFFFF803FFFFF001FFFFEA6
:10064000000FFFFC0003FFF800007FC0001F2AA876
:100650002101000001FFC00001FFC00003FFC00036
:1006600007FFC00007FFC0000FFFC0000FFFC00062
:100670001FFFC0003FFFC0003FBFC0007F3FC00062
:10068000FF3FC000FE3FC001FE3FC001FC3FC00372
:10069000F83FC007F83FC007F03FC00FF03FC01F52
:1006A000E03FC01FC03FC03FC03FC03F803FC07F52
:1006B000803FC0FF003FC0FF003FC0FFFFFFFEFFC5
:1006C000FFFFFEFFFFFFFEFFFFFFFEFFFFFFFEFF3E
:1006D000FFFFFEFFFFFFFE00003FC000003FC00025
:1006E000003FC000003FC000003FC000003FC0000E
:1006F000003FC000003FC000003FC01D2BAC2102E6
:10070000FF7FFFFFE07FFFFFE07FFFFFE07FFFFF56
:10071000E07FFFFFE07FFFFFE07FFFFFE07F8000E3
:10072000007F8000007F8000007F8000007F8000CD
:10073000007F8000007F8000007F8000007F87F8BE
:10074000007F9FFE007FFFFF807FFFFFC07FFFFFD6
:10075000C07FFFFFE07FF03FF07FC01FF07F800F82
:10076000F07F800FF87F0007F8000007F80000070F
:10077000F8000007F8000007F8000007F80000077D
:10078000F0FF000FF0FF000FF0FF001FF0FF803FB1
:10079000E07FE0FFC07FFFFFC03FFFFF801FFFFF44
:1007A000000FFFFC0003FFF800007FC0001D2CB00D
:1007B0002102FF000FF000007FFC0000FFFF00039C
:1007C000FFFF8007FFFFC007FFFFE00FFC3FE01FB8
:1007D000F00FF01FE00FF03FC007F83FC007F83FF1
:1007E0008000007F8000007F8000007F8000007F0D
:1007F000000000FF03F800FF1FFE00FF3FFF00FFA7
:100800007FFF80FFFFFFC0FFFFFFE0FFF83FF0FF2B
:10081000E01FF0FFC00FF0FFC00FF8FF8007F8FFE8
:100820008007F8FF8007F8FF8007F8FF8007F87F50
:100830008007F87F8007F87F8007F07FC00FF03FC8
:10084000C00FF03FE01FE01FF83FE01FFFFFC00FA9
:10085000FFFF8007FFFF0003FFFE0000FFF800001E
:100860003FC0001C2AA8210300FFFFFFF0FFFFFF8D
:10087000F0FFFFFFF0FFFFFFF0FFFFFFF0FFFFFFC4
:10088000F0FFFFFFF000000FF000000FF000001F6E
:10089000F000001FE000003FE000003FC000007FCC
:1008A000C000007FC00000FF800000FF800001FF4B
:1008B000000001FF000001FE000003FE000003FE37
:1008C000000007FC000007FC00000FF800000FF814
:1008D00000001FF800001FF000001FF000003FE0C4
:1008E00000003FE000007FC000007FC00000FFC0AC
:1008F0000000FF800001FF800001FF000003FF00F7
:100900000003FF000003FE000007FE000007FC00DC
:10091000001D2CB02102FF003FF00001FFFE000788
:10092000FFFF800FFFFFC01FFFFFE03FFFFFF03F13
:10093000F87FF07FE01FF07FE01FF87FC00FF87FA7
:10094000C00FF87FC00FF87FC00FF87FC00FF83FCF
:10095000E01FF03FE01FF01FF87FE00FFFFFC00730
:10096000FFFF0001FFFC0000FFF80003FFFE000F87
:10097000FFFF801FFFFFC03FF03FE07FE01FE07FF1
:10098000C00FF07FC00FF0FF8007F8FF8007F8FF6F
:100990008007F8FF8007F8FF8007F8FF8007F8FF5F
:1009A000C00FF8FFC00FF87FE01FF07FF03FF07F2F
:1009B000FFFFE03FFFFFE01FFFFFC00FFFFF8003CF
:1009C000FFFE00007FF0001D2CB02102FF001FC0C1
:1009D0000000FFF80003FFFE0007FFFF000FFFFF0E
:1009E000801FFFFF803FE0FFC03FC03FE07F801FD0
:1009F000E07F801FE07F000FF0FF000FF0FF000F8F
:100A0000F0FF000FF0FF000FF8FF000FF8FF000FDE
:100A1000F8FF000FF8FF801FF87F801FF87FC03FAE
:100A2000F87FE0FFF83FFFFFF81FFFFFF81FFFF719
:100A3000F80FFFE7F803FFC7F800FE07F000000714
:100A4000F000000FF000000FF000000FF000000FAA
:100A5000E07F801FE07F801FE03F803FC03FC07F7E
:100A6000C03FE0FF801FFFFF800FFFFF0007FFFE7A
:100A70000003FFFC0001FFF000003FC000081D1D47
:100A8000130800FFFFFFFFFFFFFFFF000000000053
:100A90000000000000000000FFFFFFFFFFFFFFFF5E
:100AA00000121A00001803700390207F001A00182B
:100AB000000000000B0000FFFFFFFFFFFFFFFFFF34
:100AC000FF11103013010601C00001C00001C00079
:100AD00001C00001C00001C00001C000FFFF80FF95
:100AE000FF8001C00001C00001C00001C00001C0C2
:100AF0000001C00001C0000708080B03023E3E3E93
:100B00003E3EF0F0F00902040B010DFF80FF80056E
:100B100005050B0502F8F8F8F8F8FF11184813015D
:100B200002FFFF80FFFF80C00380C00380C00380FE
:100B3000C00380C00380C00380C00380C00380C0A6
:100B40000380C00380C00380C00380C00380C00353
:100B500080C00380C00380C00380C00380C00380C6
:100B6000FFFF80FFFF80FFFF80061818130702FCBD
:100B7000FC1C1C1C1C1C1C1C1C1C1C1C1C1C1C1CD5
:100B80001C1C1C1C1C1C1C111848130102FFFF809C
:100B9000FFFF8000038000038000038000038000CB
:100BA0000380000380000380000380000380FFFFB8
:100BB00080FFFF80C00000C00000C00000C0000037
:100BC000C00000C00000C00000C00000FFFF80FFA8
:100BD000FF80FFFF80111848130102FFFF80FFFF15
:100BE00080000380000380000380000380000380F6
:100BF0000003800003800003800003801FFF801F2C
:100C0000FF80000380000380000380000380000356
:100C100080000380000380000380FFFF80FFFF80CF
:100C2000FFFF80111848130102C00380C00380C079
:100C30000380C00380C00380C00380C00380C00362
:100C400080C00380C00380C00380FFFF80FFFF805F
:100C50000003800003800003800003800003800005
:100C600003800003800003800003800003800003F2
:100C700080111848130102FFFF80FFFF80C00000B1
:100C8000C00000C00000C00000C00000C00000C0E4
:100C90000000C00000C00000FFFF80FFFF800003D5
:100CA0008000038000038000038000038000038035
:100CB000000380000380FFFF80FFFF80FFFF8011A3
:100CC0001848130102FFFF80FFFF80C00000C00032
:100CD00000C00000C00000C00000C00000C0000054
:100CE000C00000C00000FFFF80FFFF80C00380C085
:100CF0000380C00380C00380C00380C00380C003A2
:100D000080C00380FFFF80FFFF80FFFF801018304E
:100D1000130202FFFFFFFF000700070007000700A4
:100D2000070007000700070007000700070007008B
:100D3000070007000700070007000700070007007B
:100D4000070007111848130102FFFF80FFFF80C052
:100D50000380C00380C00380C00380C00380C00341
:100D600080C00380C00380C00380FFFF80FFFF803E
:100D7000C00380C00380C00380C00380C00380C064
:100D80000380C00380C00380FFFF80FFFF80FFFF60
:100D900080111848130102FFFF80FFFF80C003800D
:100DA000C00380C00380C00380C00380C00380C034
:100DB0000380C00380C00380FFFF80FFFF8000032B
:100DC0008000038000038000038000038000038014
:100DD000000380000380FFFF80FFFF80FFFF80058E
:100DE00010100B0502F8F8F8F8F8000000000000F9
:100DF000F8F8F8F8F80710100B03023E3E3E3E3EAE
:100E00000000003E3E3E3E3EF0F0F0FFFFFFFFFFE1
:100E1000FFFFFFFFFFFFFFFFFFFFFFFFFFFFFFFFE2
:100E2000FFFFFFFFFFFFFFFFFFFFFFFFFFFFFFFFD2
:100E3000FFFFFFFFFFFFFFFFFFFFFFFFFFFFFFFFC2
:100E4000FFFFFFFFFFFFFFFFFFFFFFFFFFFFFF00B1
:100E5000090F00FD0A01E803D820FFFD0CFD0BFD82
:100E600000000009000C010B0B0904008080808049
:100E70008080800000808004030309030790909025
:100E80000608080901014848FC4848FC4848070B87
:100E90000B0901FF107C929050381412927C1007BD
:100EA0000A0A09010042A4A4481010244A4A8407EF
:100EB0000A0A09010060909090606294889462012F
:100EC0000303090407808080030C0C0903FF204002
:100ED00040808080808080404020030C0C0903FF0C
:100EE0008040402020202020204040800707070924
:100EF000010310925438549210070707090101109A
:100F00001010FE1010100205050904FDC0C040407D
:100F100080070101090104FE020202090400C0C0A9
:100F2000070A0A090100020404081010204040804A
:100F3000070A0A0901003844828282828282443888
:100F4000070A0A090100103050901010101010FE0E
:100F5000070A0A0901007C8282040810204080FEF2
:100F6000070A0A090100FE0204081C020202827C30
:100F7000070A0A090100040C14244484FE04040432
:100F8000070A0A090100FE8080BCC2020202827CBC
:100F9000070A0A0901003C408080BCC28282827C30
:100FA000070A0A090100FE020404080810102020A4
:100FB000070A0A09010038448244384482824438CE
:100FC000070A0A0901007C828282867A020204787A
:100FD000020707090400C0C0000000C0C0020A0ADE
:100FE0000904FDC0C0000000C0C0404080050A0ADE
:100FF00009020008102040808040201008070404E7
:10100000090102FE0000FE050A0A090200804020D4
:1010100010080810204080070A0A0901007C82821B
:1010200002040810100010070A0A0901007C8282DD
:101030009EA2A69A80807C070A0A09010010284413
:10104000828282FE828282070A0A090100F8848273
:1010500084F884828284F8070A0A0901007C82806D
:101060008080808080827C070A0A090100F88482DF
:10107000828282828284F8070A0A090100FE808047
:1010800080F880808080FE070A0A090100FE8080C7
:1010900080F88080808080070A0A0901007C8280B5
:1010A00080808E8282827C070A0A09010082828205
:1010B00082FE8282828282050A0A090200F82020CA
:1010C000202020202020F8080A0A0901001F04041B
:1010D00004040404048478070A0A0901008284884D
:1010E00090E0A090888482070A0A0901008080802D
:1010F000808080808080FE070A0A0901008282C603
:10110000AAAA9292828282070A0A0901008282C2F6
:10111000A2928A86828282070A0A0901007C828260
:101120008282828282827C070A0A090100FC828212
:1011300082FC8080808080070C0C0901FE7C82820A
:1011400082828282A2927C0806070A0A090100FCB8
:10115000828282FC9088848282070A0A0901007CCC
:10116000828280700C0282827C070A0A090100FEDA
:10117000101010101010101010070A0A0901008238
:1011800082828282828282827C070A0A090100822C
:10119000828244444428282810070A0A0901008250
:1011A00082828292929292AA44070A0A09010082DC
:1011B000824428101028448282070A0A090100820A
:1011C000824428101010101010070A0A090100FEAE
:1011D0000204081020408080FE040C0C0903FFF07C
:1011E00080808080808080808080F0070A0A0901EA
:1011F0000080404020101008040402040C0C090276
:10120000FFF010101010101010101010F007040450
:10121000090106102844820801010900FFFF0303A9
:10122000030903088040200707070901007C020228
:101230007E82867A070A0A090100808080BCC28209
:101240008282C2BC0707070901007C8280808082FD
:101250007C070A0A0901000202027A8682828286DB
:101260007A0707070901007C8282FE80807C070ADA
:101270000A0901001C22222020F820202020070A31
:101280000A0901FD7A84848478807C82827C070A42
:101290000A090100808080BCC28282828282050AA3
:1012A0000A090200600000E02020202020F8060D3E
:1012B0000D0901FD0C00001C040404040484848452
:1012C00078070A0A090100808080828CB0C0B08C47
:1012D00082050A0A090200E0202020202020202088
:1012E000F8070707090100EC929292929282070791
:1012F00007090100BCC282828282820707070901B6
:10130000007C82828282827C070A0A0901FDBCC2BB
:10131000828282C2BC808080070A0A0901FD7A8627
:10132000828282867A0202020707070901009C6214
:1013300042404040400707070901007C82807C0250
:10134000827C0709090901002020FC20202020229E
:101350001C0707070901008484848484847A0707B2
:101360000709010082824444282810070707090161
:10137000008282929292AA440707070901008244E0
:101380002810284482060A0A0901FD848484848482
:101390008C74048478070707090100FE04081020F4
:1013A00040FE050C0C0903FF3840404020C0C0201F
:1013B00040404038010C0C0904FF80808080808010
:1013C000808080808080050C0C0901FFE0101010E7
:1013D00020181820101010E007030309010762927B
:1013E0008CFFFFFFFFFFFFFFFFFFFFFFFFFFFFFF80
:1013F000FFFFFFFFFFFFFFFFFFFFFFFFFFFFFFFFFD
:10140000FFFF00000009000C010B0B0904008080A5
:101410000000808080808080800608080901000824
:10142000789490A0A47840070A0A0901001C2220A1
:1014300020F8202060A25C070606090103827C4494
:10144000447C82070A0A090100828244287C107CBD
:10145000101010010B0B0904FF8080808080008039
:1014600080808080040B0B0902FF60908060909068
:101470009060109060050202090209888808090935
:101480000900013C4299A5A1A599423C050707091D
:101490000103609070907800F807080809010112B4
:1014A00024489090482412060404090102FC040414
:1014B00004050101090204F80809090900013C4278
:1014C000B9A5B9A9A5423C060101090109FC04041A
:1014D00004090306609090600709090901011010D2
:1014E00010FE10101000FE040606090104609010A2
:1014F0006080F004060609010460902010906003EB
:1015000003030903082040800709090901FE8282BC
:10151000828282C6BA8080070A0A0901007E8A8A0E
:101520008A7A0A0A0A0A0A020202090404C0C004EA
:1015300003030902FD30906003060609010440C060
:10154000404040E00506060901047088887000F8F4
:101550000708080901019048241212244890070A3C
:101560000A09010040C0404042E60A121A06070A72
:101570000A09010040C040404CF2020C101E070A4C
:101580000A0901006090201092660A121A06070AE2
:101590000A0901001000101020408082827C070C94
:1015A0000C0901004020100038448282FE828282B1
:1015B000070C0C0901000408100038448282FE82E6
:1015C0008282070C0C0901001028440038448282F2
:1015D000FE828282070B0B090100629C0038448264
:1015E00082FE828282070B0B0901004444003844CA
:1015F0008282FE828282070B0B0901003844382860
:10160000448282FE828282070A0A0901006E90905B
:101610009090FC9090909E070D0D0901FD7C8280BA
:101620008080808080827C184830070C0C09010083
:1016300040201000FE404078404040FE070C0C095E
:10164000010004081000FE404078404040FE070CB6
:101650000C09010010284400FE404078404040FE44
:10166000070B0B090100444400FE40407840404015
:10167000FE050C0C09020080402000F820202020EC
:101680002020F8050C0C09020008102000F820208A
:1016900020202020F8050C0C09020020508800F8BA
:1016A000202020202020F8050B0B0902008888004C
:1016B000F8202020202020F8080A0A0900007C4297
:1016C0004141E1414141427C070B0B090100629C11
:1016D0000082C2A292928A8682070C0C0901004005
:1016E0002010007C8282828282827C070C0C09019D
:1016F00000040810007C8282828282827C070C0CAB
:10170000090100102844007C8282828282827C0748
:101710000B0B090100629C007C8282828282827CA7
:10172000070B0B0901004444007C82828282828282
:101730007C07070709010182442810284482070C0E
:101740000C0901FF027C868A8A9292A2A2C27C8046
:10175000070C0C09010040201000828282828282E4
:10176000827C070C0C09010004081000828282822E
:101770008282827C070C0C090100102844008282BE
:1017800082828282827C070B0B0901004444008222
:101790008282828282827C070C0C0901000408107C
:1017A000008282442810101010070A0A09010080E4
:1017B00080FC828282FC808080060A0A090100384F
:1017C000444448D04844444458070B0B09010020C6
:1017D0001008007C02027E82867A070B0B0901004A
:1017E000040810007C02027E82867A070B0B090136
:1017F00000102844007C02027E82867A070A0A09C9
:101800000100324C007C02027E82867A070A0A09B5
:1018100001004444007C02027E82867A070B0B0999
:101820000100182418007C02027E82867A070707CE
:101830000901006C92127C90926E070A0A0901FD60
:101840007C82808080827C184830070B0B09010065
:10185000402010007C8282FE80807C070B0B0901F7
:1018600000040810007C8282FE80807C070B0B093C
:101870000100102844007C8282FE80807C070A0AD6
:101880000901004444007C8282FE80807C050B0BB1
:1018900009020080402000E02020202020F8050BD5
:1018A0000B09020010204000E02020202020F80634
:1018B0000B0B090100205088007010101010107CD4
:1018C000050A0A090200909000E02020202020F85C
:1018D000070B0B090100483050087C82828282820B
:1018E0007C070A0A090100629C00BCC282828282D3
:1018F00082070B0B090100402010007C828282824B
:10190000827C070B0B090100040810007C82828294
:1019100082827C070B0B090100102844007C828224
:101920008282827C070A0A090100629C007C828212
:101930008282827C070A0A0901004444007C828278
:101940008282827C07090909010010381000FE001C
:101950001038100709090901FF027C8A8A92A2A2A5
:101960007C80070B0B0901004020100084848484D4
:1019700084847A070B0B0901000408100084848416
:101980008484847A070B0B090100102844008484A6
:10199000848484847A070A0A090100484800848400
:1019A000848484847A060E0E0901FD0810200084C8
:1019B000848484848C74048478070C0C0901FD8071
:1019C0008080BCC28282C2BC808080060D0D09016D
:1019D000FD48480084848484848C740484780729B6
:1019E00011241FBECFEFD8E0DEBFCDBF13E0A0E0D3
:1019F000B1E0E0EAF9E502C005900D92A23EB10720
:101A0000D9F725E0A2EEB3E001C01D92A332B207E0
:101A1000E1F71CE0C0EFDCE004C02197FE010E946A
:101A2000C82CCF3ED107C9F70E941A200C94CE2CA7
:101A30000C9400004F925F926F927F928F929F92D0
:101A4000AF92BF92CF92DF92EF92FF920F931F93CC
:101A5000CF93DF9300D000D0CDB7DEB74B015C0150
:101A600029013A016701780120E030E0A9010E94D4
:101A7000E22A87FDA6C020E030E0A901C301B2013F
:101A80000E94E22A87FD9DC020E030E0A901C80144
:101A9000B6010E94E22A87FD94C081E02091C30430
:101AA0003091C4042130310509F080E08093E404D2
:101AB0008092A9049092AA04A092AB04B092AC04C4
:101AC0004092AD045092AE046092AF047092B004A4
:101AD000C092B104D092B204E092B304F092B40484
:101AE0006091D7047091D8048091D9049091DA0460
:101AF0000E948F2B20E030E04AE754E40E94E72A5E
:101B000069837A838B839C838092B5049092B60418
:101B1000A092B704B092B8049B01AC01C301B2011A
:101B20000E94462C2B013C014092B9045092BA0409
:101B30006092BB047092BC0429813A814B815C8124
:101B4000C701B6010E94E72A6B017C01C092BD0467
:101B5000D092BE04E092BF04F092C0048091C10410
:101B60009091C204019769F5A501940160E070E0CD
:101B7000CB010E94752A6093B5047093B6048093DC
:101B8000B7049093B804A301920160E070E0CB0128
:101B90000E94752A6093B9047093BA048093BB04C1
:101BA0009093BC04A701960160E070E0CB010E9415
:101BB000752A6093BD047093BE048093BF04909314
:101BC000C0040F900F900F900F90DF91CF911F9155
:101BD0000F91FF90EF90DF90CF90BF90AF909F90CC
:101BE0008F907F906F905F904F90089580E0089560
:101BF0002091ED043091EE042817390799F1909364
:101C0000EE048093ED04009739F120910005FC016A
:101C1000211129C03596E491E09301050C96FC0151
:101C200084918093020580910105082E000C990B88
:101C300020910205821B910927FD939520910305B0
:101C4000203441F0829FC001112426E096958795AB
:101C50002A95E1F78093040586EF9DE09093FF04B9
:101C60008093FE040895213031F43F96E491E0938F
:101C700001054096D4CF3D96E491E09301050E9680
:101C8000CECFFC01808D8F5F0895833081F028F4E2
:101C9000813099F08230A9F008958730A9F088301A
:101CA000C9F08430B1F4809180008F7D03C08091B1
:101CB00080008F7780938000089584B58F7784BDEE
:101CC000089584B58F7DFBCF8091B0008F7780938E
:101CD000B00008958091B0008F7DF9CFCF93DF934E
:101CE000282F30E0F901E255FE4F8491F901E656C4
:101CF000FE4FD491F901EA57FE4FC491CC23A1F0D5
:101D000081110E94450EEC2FF0E0EE0FFF1FE4580A
:101D1000FE4FA591B491EC91ED2381E090E009F4A0
:101D200080E0DF91CF91089580E090E0FACF1F939B
:101D3000CF93DF93282F30E0F901E255FE4F8491D5
:101D4000F901E656FE4FD491F901EA57FE4FC491CE
:101D5000CC23A9F0162F81110E94450EEC2FF0E044
:101D6000EE0FFF1FEE58FE4FA591B4918FB7F89478
:101D7000EC91111108C0D095DE23DC938FBFDF9169
:101D8000CF911F910895DE2BF8CFCF93DF9390E092
:101D9000FC01E656FE4F24918A579E4FFC01849128
:101DA0008823C9F090E0880F991FFC01E859FE4F85
:101DB000A591B491FC01EE58FE4FC591D4916111EB
:101DC0000DC09FB7F8948C91209582238C938881C5
:101DD000282328839FBFDF91CF910895623051F46B
:101DE0009FB7F8943C91822F809583238C93E88150
:101DF0002E2BEFCF8FB7F894EC912E2B2C938FBF17
:101E0000EACFCF93DF93EC0161E089E00E94C50E39
:101E1000209731F460E089E0DF91CF910C94970E28
:101E2000CF3FD10511F461E0F6CFE7EBF1E0E491AB
:101E3000E33029F140F4E130B1F0E230D9F0C038BC
:101E4000D1058CF7E7CFE73021F1E83051F1E430EC
:101E5000B1F780918000806280938000D0938B00E6
:101E6000C0938A0004C084B5806884BDC7BDDF917B
:101E7000CF91089584B5806284BDC8BDF8CF8091AC
:101E80008000806880938000D0938900C093880090
:101E9000EECF8091B00080688093B000C093B30013
:101EA000E6CF8091B00080628093B000C093B40010
:101EB000DECF3FB7F8948091A3049091A404A09141
:101EC000A504B091A60426B5A89B05C02F3F19F024
:101ED0000196A11DB11D3FBFBA2FA92F982F8827AA
:101EE000BC01CD01620F711D811D911D42E0660F85
:101EF000771F881F991F4A95D1F708958F929F9257
:101F0000AF92BF92CF92DF92EF92FF924B015C01B2
:101F10000E94590F6B017C010E94590F6C197D09B9
:101F20008E099F09683E734081059105A8F321E061
:101F3000821A9108A108B10888EEC80E83E0D81E65
:101F4000E11CF11C81149104A104B10429F7FF9054
:101F5000EF90DF90CF90BF90AF909F908F900895BB
:101F60002FB7F89460919F047091A0048091A10410
:101F70009091A2042FBF0895AF92BF92CF92DF92AB
:101F8000EF92FF920F931F93CF93DF936C017B012E
:101F90008B01040F151FEB015E01AE18BF08C017BF
:101FA000D10759F06991D601ED91FC910190F08132
:101FB000E02DC6010995892B79F7C501DF91CF91F5
:101FC0001F910F91FF90EF90DF90CF90BF90AF9057
:101FD00008950895DC011696ED91FC9117971296DD
:101FE0008C91481B477081E090E001C0880F4A95B2
:101FF000EAF7E60FF11D3081222319F0832B80834D
:10200000089580958323FBCFFB014181DC0112966B
:102010002C911297421768F013962C91139724175E
:1020200040F0608115962C91621718F424810C946D
:10203000EA0F0895FC0180819281980F928321819B
:10204000921760F494819F5F94839381890F821724
:1020500010F08FEF820F838381E0089580E0089570
:10206000FC01128280818150838314820895DB01F8
:10207000ED91FC9109940F931F93CF93DF931F92DF
:10208000CDB7DEB70091EB041091EC04E0911A0596
:10209000F0911B0582E0099530E020E04AE0B801AC
:1020A00089EE94E00E943710182FE0911A05F09104
:1020B0001B0583E00995E0911A05F0911B0580E06E
:1020C00009951123B9F16091EB047091EC049E0124
:1020D0002F5F3F4F46E489EE94E00E9437108981DC
:1020E0008093E9046091EB047091EC049E012F5FF2
:1020F0003F4F47E489EE94E00E9437108981809336
:10210000EA046091EB047091EC0430E020E048E4D4
:1021100089EE94E00E9437108093F4046091EB0400
:102120007091EC042CE135E047E189EE94E00E94E7
:10213000371011E0812F0F90DF91CF911F910F91F8
:102140000895CF93DF9380912205811105C081E02E
:10215000809322050E943B10C091EB04D091EC04C7
:10216000E0911A05F0911B0582E00995E0911A05AE
:10217000F0911B0581E0099530E020E044E1BE01CB
:1021800089EE94E00E9437102CE135E047E1BE0172
:1021900089EE94E00E943710E0911A05F0911B053A
:1021A00080E0DF91CF9109940F931F93CF93E0913B
:1021B000F704F091F804309719F089EE94E009954E
:1021C0000091EB041091EC04E0911A05F0911B05CD
:1021D00082E00995E0911A05F0911B0581E00995CF
:1021E00030E020E045E1B80189EE94E00E9437102C
:1021F000C82F882341F02CE135E047E1B80189EE92
:1022000094E00E943710E0911A05F0911B0580E0E0
:1022100009958C2FCF911F910F9108950B96FC017A
:10222000849108950A96FC0184910895FC0184919B
:1022300008950E941611882321F0823011F083E066
:10224000089586E00895FC01E60FF11D849190E069
:10225000982F88273196E4918E0F911D089568E09C
:102260000C94231166E00C9423115F926F927F927D
:102270008F929F92AF92BF92CF92DF92EF92FF9296
:102280000F931F93CF93DF93EC01E62EF42EC22E13
:102290000C811D81C8010E941611D82E8C819D8150
:1022A0000E941911982E21E0AA24AA94D21202C0E9
:1022B0002FE0A22E8C819D810E941211D82E8C813C
:1022C0009D810E940E11B82E8C819D810E942F113C
:1022D000E0E6EC1578F4009769F0080F191F91E615
:1022E000D92EBC14C0F4188A1B8A1C8A198A1A8A2F
:1022F00080E0A0C08C819D810E943211F0E4FC1529
:1023000038F4009729F0080F191F81E4D82EE9CF7F
:102310000F5E1F4FE6CFBD1430F3892D90E0F8011A
:1023200024912F3F31F40F5F1F4FBD14E1F2D3947E
:10233000F6CFCD1072C08C819D810E94161198013C
:102340002F5F3F4FF801882319F0823009F04EC00B
:1023500084918B8BF90124912C8BF8013396E491B5
:10236000E88BF8013496E491E98BF8013596E49115
:10237000EA8B0115110509F4BBCF8C819D810E9468
:1023800019113C89F31A9A89F91A9FEF930F9F0D3F
:102390002CA94EA94F1508F449C0921718F49F159F
:1023A00008F047C02B899989E90E9FEF920F9E0D87
:1023B0004BA95DA95E1508F44DC0941718F49E153D
:1023C00008F037C0080F111D295F722E769476949D
:1023D00076946F2C630E5E01FCE1AF0EB11C872C6E
:1023E000912CF61431F15E2C68014AC08491982F2B
:1023F0009F7092509A8B82958F70898BF9012491EE
:10240000822F8F708C8B22952F702B8BF801329638
:10241000E491E295EF70E88BACCF3296E491EA213B
:10242000E80FF92FF11D0E0F1F1F7FCF921708F035
:10243000B6CF8889DF91CF911F910F91FF90EF90D8
:10244000DF90CF90BF90AF909F908F907F906F90D4
:102450005F900895941708F0B2CFEBCFF601849106
:102460006A817B815C8EFD8E1F8E8E8F95014BE382
:10247000CE010E943710FFEFCF1ADF0A28E0520E7C
:102480008C2D801B871550F3080D191DF394A9CFCF
:10249000EF92FF920F931F93CF93DF93F82E062FA7
:1024A000E42E152FE091FE04F091FF0489EE94E0F4
:1024B0000995080FCE2DD12F10E02991211108C0C8
:1024C000812FDF91CF911F910F91FF90EF90089591
:1024D000402F6F2D89EE94E00E943511F80E180FF1
:1024E000ECCF0F931F93CF93DF938C01E091FE0409
:1024F000F091FF0489EE94E00995D82FC0E0F8012F
:102500002491222351F04D2F6C2F89EE94E00E94EC
:102510003511C80F0F5F1F4FF2CF8C2FDF91CF9176
:102520001F910F9108952EE93FE0009709F4089557
:10253000F9013197F1F70197F8CFCF93DF9300D0EE
:10254000CDB7DEB720ED37E03A8329839091BC0008
:10255000982311F081E00FC029813A81232B81F467
:102560008091A80481FDF6CF8091A70481110DC050
:1025700091E09093A7040F900F90DF91CF91089571
:1025800029813A8121503109DFCF80E0F4CF84EAFC
:102590008093BC0061E080E80E949D12811102C01E
:1025A00080E008958091B900887F883051F08031B3
:1025B00041F08091A7048111F3CF82E08093A704BA
:1025C000EFCF88E78093BB0084E88093BC0062E093
:1025D00080E80E949D12882319F38091A80481FD50
:1025E00005C08091B900887F883119F781E008958E
:1025F00084E98093BC0064E080E10C949D12809398
:10260000BB0084E88093BC0063E080E80E949D12D8
:102610008823A1F08091A80481FD0DC08091B900AC
:10262000887F883241F08091A704811106C092E032
:102630009093A704089581E0089580E00895109292
:10264000A70408958093A8041092B90084FF05C0E0
:102650008CE08093B8000C941F1388E4FACFCF93DA
:10266000DF93FC0123A5222389F0EC010E94C7120D
:10267000811104C080E0DF91CF9108958EA1811176
:1026800007C00E94FF128823A9F31BA681E0F3CFA5
:1026900080E4F7CF0F931F93CF93DF93C62FD42FF0
:1026A0008901633001F138F4613099F0623009F446
:1026B00049C0C1E012C0663029F1673091F1653040
:1026C000C1F70E942F13811117C00E94F812C0E0B9
:1026D00004C0FC0186A50E9422138C2FDF91CF91AC
:1026E0001F910F910895FC0116A221E023A741112B
:1026F000E0CF0E94F812DDCF8D2F0E94FF128111D2
:10270000D8CFE3CF0E942F138823F9F2DD2389F27B
:10271000F80181918F010E94FF128823B1F2D150FC
:10272000F5CF0E942F13882381F2DD2311F2F801E7
:1027300084910E94FF12C82F882379F20F5F1F4FE8
:10274000D150F3CFFC0146A321E023A7B2CFDB0198
:102750001496ED91FC9130E020E065E00994DB01F6
:102760001496ED91FC9130E020E062E00994DB01E9
:102770001496ED91FC9130E020E063E00994CF9253
:10278000DF92EF92FF920F931F93CF93DF938C0111
:102790007B016A0180E0F601C491811110C081E0E3
:1027A000CF3F49F04C2FB701C8010E94A7138823DF
:1027B00009F444C080E0BFEFCB1ADB0AECCF4FEF47
:1027C000CF3F89F3CE3FD9F1C03FA0F7C03E38F0EC
:1027D0004C2F4F70B701C8010E94AF13EBCFC03D23
:1027E00038F04C2F4F70B701C8010E94B713E2CFE9
:1027F000C03CF8F0D7011496ED91FC9130E020E058
:1028000040E064E0C8010995C295C07FCE5FD0E08A
:10281000CE010E949312D7011496ED91FC9130E005
:1028200020E041E064E0C8010995CE010E949312C6
:10283000C1CFC7FDBFCF8C2F90E0F8CF80E0DF91F4
:10284000CF911F910F91FF90EF90DF90CF9008955F
:10285000AF92BF92CF92DF92FF920F931F93CF93CD
:10286000DF936C018B01F42EE90180E1481709F434
:102870007EC0841778F1AAE04A1709F461C0BFE06E
:102880004B1709F47FC0F80102811381F2E3FF16B0
:1028900009F4DDC0FF1508F48EC085E1F81609F4CF
:1028A000DBC0A7E1FA1609F4ECC0B4E1FB1265C085
:1028B000D8011696ED91FC91179715968C918E0F75
:1028C0009F2F911D11928E179F07E1F7C8010E945B
:1028D000301053C0E1E14E1709F451C0F5E14F1338
:1028E000D2CFFB01A280B38047E950E0C6010E942D
:1028F000BF13D50114964C91406BB801C6010E94DC
:10290000A71341E0B801C6010E94AF13F50126816B
:102910003781D8011496ED91FC91D50115964C9113
:1029200066E0C601099581111CC080E0DF91CF915E
:102930001F910F91FF90DF90CF90BF90AF900895BF
:10294000DB011496ED91FC9130E020E042E061E083
:10295000C60109954FE950E0B801C6010E94BF13B6
:1029600092CF40E0B801C6010E94B7138CCF4EE869
:1029700050E0B801C6010E94BF1381E0D7CF43E801
:1029800050E0F7CF41E0C6010E94B71340E0B80124
:10299000C6010E94AF1341E8B801C6010E94A71307
:1029A0004881B801C6010E94A71340E0B801C601E2
:1029B0000E94B713E2CFE6E4FE1609F46CC0F7E418
:1029C000FF1609F46DC08BE3F812D7CF99818B8184
:1029D00038E0390F813031F0833011F0392F02C0E7
:1029E000392F985021E0D80113964C91491708F4DB
:1029F00020E041E0391708F040E091E0F801528111
:102A0000351708F490E0322F342B932319F4242344
:102A100009F4B3CFFA80D12CC12C843048F490E073
:102A2000FC01EA5EFD4FC0808E5E9D4FDC01DC90B4
:102A3000F7FE04C0BE01C8010E94041088818C0DFD
:102A4000888389818D0D8983FF0C91F796CFBE0114
:102A5000C8010E94041091CFC8010E941A10882357
:102A600009F463CFD8011696ED91FC91179715964E
:102A70008C918E0F9F2F911D11928E179F07E1F75A
:102A80007CCF1882F80182818983858181508A8375
:102A900083818B8372CFD80115968C9188836DCFFB
:102AA000F8018181FBCF80917A00806980937A0060
:102AB0008EE480937C0061E070E080E090E00E9412
:102AC0007E0F83B7817F826083BF80E130E020E0AA
:102AD00093B7916093BF889593B79E7F93BF909172
:102AE0007A0096FDFCCF4091780050917900240F38
:102AF000351F815069F780917A008F7780937A0033
:102B000084E0369527958A95E1F750E040E064EB44
:102B10007BE281E190E00E941A2AC9010895809128
:102B20007A00806980937A0088EC80937C0064E16D
:102B300070E080E090E00E947E0F83B7817F82602A
:102B400083BF80E270E060E093B7916093BF8895A7
:102B500093B79E7F93BF90917A0096FDFCCF209112
:102B6000780030917900620F731F815069F780916E
:102B70007A008F7780937A0076956795769567953A
:102B800062527A4090E080E00E948F2B26EF38E27C
:102B90004CE151E40E94E72A089590917A009069EF
:102BA00090937A008E50806480937C0083B7817FFD
:102BB000826083BF20E290E080E033B7316033BFB2
:102BC000889533B73E7F33BF30917A0036FDFCCF16
:102BD0004091780050917900840F951F215069F73A
:102BE00020917A002F7720937A0025E0969587959B
:102BF0002A95E1F708958FE00E94CD15A0916E040B
:102C0000B0916F049C010E94662A0E94912B28E5D6
:102C100039E743E353E40E94E72A0E94602BCB018B
:102C200008950F931F93CF938091B101882399F05A
:102C3000CFEF0FEE11E061E085E00E94970EC80132
:102C40000197F1F760E085E00E94970EC8010197B7
:102C5000F1F7C15081F7CF911F910F910895CF9255
:102C6000DF92EF92FF920F931F93CF93DF93D82EB3
:102C7000C92E86E00E946E0EC1E0892B09F0C0E0EB
:102C80000E94A11081E4E82E8EE0F82E8FE49EE0F1
:102C90000E94F80DF092FF04E092FE040D2D1C2D11
:102CA000D0E0F801419151918F016D2F80E00E9499
:102CB0004812D05FD038A9F70E94D4108111E6CF16
:102CC000CC2369F086E00E946E0EC1E0892B39F0BA
:102CD0006AE070E080E090E00E947E0FC0E086E055
:102CE0000E946E0E892B61F7C111ECCFDF91CF915D
:102CF0001F910F91FF90EF90DF90CF900C941116E1
:102D00002F923F924F925F926F927F928F929F92FB
:102D1000AF92BF92CF92DF92EF92FF920F931F93E9
:102D2000CF93DF9300D000D0CDB7DEB77C01942ED7
:102D3000FC012080318077247394411101C0712CF3
:102D400070E0759567956A8310927504109274040B
:102D500062507109660F771F709373046093720459
:102D600081E090E09093710480937004892D90E04D
:102D7000880F991F9093800480937F0486E00E94BF
:102D80006E0E66246394892B09F0612CCC24CA94BE
:102D90004FE7D42E51E4A52E5EE0B52E80917F043E
:102DA00090918004959587959C838B835B808C01A3
:102DB0001127C801870D911D77FC9A9589199109F2
:102DC000712C97FD06C08330910514F082E090E0ED
:102DD000782E0E94A110272D072C000C330BC9015F
:102DE0000196E82FE295E07FE9832C9DC0012D9D9F
:102DF000900D3C9D900D1124080F191F000F111FFD
:102E00008FE49EE00E94F80DB092FF04A092FE04B1
:102E1000F7014081518160E080E00E944812FAE1B0
:102E20002F16F2E03F0661F440918D0486E0489F42
:102E3000A00111244B525E4F60E086E30E944812CD
:102E40004FE152E0698180E00E9448128824839417
:102E5000912C412C4394852D840D87199A818917D3
:102E600078F4F401EE0FFF1FE00FF11FEE0DFF1DD0
:102E700040815181642D6295607F8CE00E944812F0
:102E8000EFEF8E1A9E0AF3E04F12E4CF0E94D410A7
:102E90008111B6CF662061F086E00E946E0E892B0C
:102EA00039F06AE070E080E090E00E947E0F612CD3
:102EB00086E00E946E0E892BE1F461101AC00E9418
:102EC0001116852D0F900F900F900F90DF91CF91DD
:102ED0001F910F91FF90EF90DF90CF90BF90AF9038
:102EE0009F908F907F906F905F904F903F902F902A
:102EF00008959B8053CF3F924F925F926F927F9243
:102F00008F929F92AF92BF92CF92DF92EF92FF92F9
:102F10000F931F93CF93DF93CDB7DEB72E970FB6E6
:102F2000F894DEBF0FBECDBF80919704882309F4CB
:102F3000A5C110929A0410929B0410929C041092C6
:102F40009D0480909A0490909B04A0909C04B09063
:102F50009D04C0908804D0908904E0908A04F09089
:102F60008B04A7019601C501B4010E94752A2B01AB
:102F70003C0120E030E0A9010E94412C18160CF021
:102F8000A0C1C301B2010E94602B8091BE018823C1
:102F900009F4B8C1C0926304D0926404E09265045D
:102FA000F0926604E12CF12C00EA10E420E030E01D
:102FB00040E450E46E31710540F0E12CF12C00E862
:102FC0001FE320E030E040E05FE360E070E080E39A
:102FD00091E40E941A0D8091E304882309F42AC128
:102FE0000E94B00F6D837E838F8398878091CB047E
:102FF0009091CC04A091CD04B091CE044D815E811E
:103000006F817885481B590B6A0B7B0B8091D70425
:103010009091D804A091D904B091DA0448175907C7
:103020006A077B0708F406C1E091C504F091C60465
:1030300080819181A281B38189839A83AB83BC8390
:10304000E091C904F091CA049C01AD0160817181D5
:10305000828193810E94752A4B015C012091D304E7
:103060003091D4044091D5045091D60469817A817D
:103070008B819C810E94752A6B017C012091B9048F
:103080003091BA044091BB045091BC04C501B40115
:103090000E94462C2091CF043091D0044091D1045D
:1030A0005091D2040E94762A2B013C014092CF0419
:1030B0005092D0046092D1047092D2043090E40413
:1030C00031101AC02091B5043091B6044091B70474
:1030D0005091B804C701B6010E94462C9B01AC0177
:1030E000C301B2010E94752A6093CF047093D0048B
:1030F0008093D1049093D2044090CF045090D00498
:103100006090D1047090D2041091DF049091E0049B
:103110009E87A091E104AD870091E204212F392F11
:103120004A2F502FC301B2010E94412C18160CF0F7
:10313000CCC0812F9E85AD85B02F8093CF04909316
:10314000D004A093D104B093D204332009F4D6C0A4
:103150002091B5043091B6044091B7045091B80461
:10316000C501B4010E94462C4B015C012091BD04B5
:103170003091BE044091BF045091C004C701B60114
:103180000E94462C9B01AC016091CF047091D00449
:103190008091D1049091D2040E94752AA5019401D6
:1031A0000E94762A6B017C019B01AC01612F7E8518
:1031B0008D85902F0E94E22A87FD18C01091DB04B4
:1031C0009091DC049E87A091DD04AD870091DE0420
:1031D000212F392F4A2F502FB601C7010E94E22A12
:1031E00087FD04C01C2DDE86ED860F2DE091C704FF
:1031F000F091C804812F9E85AD85B02F8083918387
:10320000A283B38389819A81AB81BC818093D304EB
:103210009093D404A093D504B093D6048D819E815D
:10322000AF81B8858093CB049093CC04A093CD0458
:10323000B093CE04609191047091920480919304B4
:10324000909194040E94592BCB012E960FB6F894BE
:10325000DEBF0FBECDBFDF91CF911F910F91FF90C9
:10326000EF90DF90CF90BF90AF909F908F907F9026
:103270006F905F904F903F900C94010F8091960457
:10328000609183017091840181110EC08091860448
:103290009091870420919504BC01222329F060912C
:1032A0007E01680F792F711D90E080E00E948F2BC6
:1032B00060939A0470939B0480939C0490939D0464
:1032C00040CEC301B20190585ECE8091DB04909154
:1032D000DC04A091DD04B091DE0489879A87AB8776
:1032E000BC879C01AD01C301B2010E94E22A87FFA5
:1032F0002CCF89859A85AB85BC851FCF812C912CDD
:10330000540134CF20E030E040E05FE3C701B60174
:103310000E94762A9B01AC01C501B4010E94412C98
:1033200018164CF410929104109292041092930487
:10333000109294047FCF80E090E0AFE7B3E48093F5
:10334000910490939204A0939304B093940472CF49
:103350004F925F926F927F928F929F92AF92BF92A5
:10336000CF92DF92EF92FF92CF93DF9380906A0427
:1033700090906B04A0906C04B0906D04C0918D048B
:10338000D0E0C501B4010E94592B6B017C0120E003
:1033900030E048E453E4C501B4010E94E22A93E01E
:1033A000CC0FDD1F9A95E1F7C55DDE4F87FF31C079
:1033B0002881398150E040E0255131094109510906
:1033C000C701B6010E94B82C28EC30E040E050E084
:1033D0000E941A2ACA01B9016B5E7F4F8F4F9F4F1F
:1033E0000E94912B609388047093890480938A04CF
:1033F00090938B04DF91CF91FF90EF90DF90CF906F
:10340000BF90AF909F908F907F906F905F904F9004
:1034100008954A805B80712C612C20E030E04CE8FC
:1034200053E4C501B4010E94E22A87FF1FC08880CF
:103430009980B12CA12CA7019601285C3109410982
:103440005109C301B201681979098A099B090E94CF
:10345000B82C20E530E040E050E00E941A2ACA0172
:10346000B901680D791D8A1D9B1DBACF2C813D8144
:1034700050E040E02419350946095709C701B60153
:1034800068517140810991090E94B82C20E530E013
:1034900040E050E00E941A2ACA01B901640D751D6E
:1034A000861D971D9DCF8F929F92AF92BF92CF9214
:1034B000DF92EF92FF928FEF90E00E94010F8BEA74
:1034C00094E00197F1F78EE00E94CD157C018AE02F
:1034D0000E946E0E90916204981729F091E09093EB
:1034E0008C0480936204809108019FEF980F909361
:1034F0000801811106C00E94FB1590938F048093F0
:103500008E04609191047091920480919304909143
:1035100094040E94592BCB010E94010F80906A04F1
:1035200090906B04A0906C04B0906D04B70190E093
:1035300080E00E948F2BA50194010E94752A2DEC3A
:103540003CEC4CE45DE30E94462CA50194010E94F2
:10355000762A60936A0470936B0480936C04909352
:103560006D040E94A819609198047091990490E0EC
:1035700080E00E948F2B6B017C0120919A04309196
:103580009B0440919C0450919D040E94E22A811169
:1035900064C0209188043091890440918A0450913C
:1035A0008B04C701B6010E94752A6B017C0120E0E3
:1035B00030E0A9010E94412C18160CF044C020E014
:1035C00030E040E450E4C701B6010E94412C1816D7
:1035D0000CF443C0609186047091870490E080E011
:1035E0000E948F2B209188043091890440918A0495
:1035F00050918B040E94752A6B017C0120E030E021
:10360000A9010E94412C1816BCF5C701B6010E9401
:10361000602B65307105A0F580910502811105C010
:103620008091D40181110E94111681E080930502DE
:103630001092D401FF90EF90DF90CF90BF90AF90A9
:103640009F908F90089520E030E040E450ECC70157
:10365000B6010E94E22A87FFBDCF60918804709175
:10366000890480918A0490918B040E94602B70934E
:10367000990460939804AECFC701B6019058C7CFA4
:1036800010920502D7CFDF92EF92FF920F931F9314
:10369000CF93DF93EC01D62E1CAD0BAD7C0184E003
:1036A000E80EF11CE98DFA8DC7010995412F480FED
:1036B0002D2D602FC7010E9435119BAD890F8BAF57
:1036C00081E090E0DF91CF911F910F91FF90EF90FB
:1036D000DF9008950F931F93CF93DF938C01D0E079
:1036E000C0E0F801EC0FFD1F6491662341F085EE08
:1036F00094E00E94431B892B11F02196F2CFCE015A
:10370000DF91CF911F910F910895682F85EE94E07E
:103710000C94431B2F923F924F925F926F927F9235
:103720008F929F92AF92BF92CF92DF92EF92FF92D1
:103730000F931F93CF93DF9300D01F92CDB7DEB7C7
:10374000412C1B821A820EE310E040ECE42EF12C97
:10375000CC24C394D12C60E2262E7EEB872E912CB4
:103760008A81898386E00E946E0E33243394892BEC
:1037700009F0312C1093750400937404F0927304D3
:10378000E0927204D0927104C0927004E2E8F0E01A
:10379000F0938004E0937F0431E4A32E3EE0B32E47
:1037A00080917F049091800495958795582EFFE134
:1037B0008F1342C01093750400937404F092730445
:1037C000E0927204D0927104C092700490928004CE
:1037D00080927F049FE5592E0E94A1108FE49EE005
:1037E0000E94F80DB092FF04A092FE0484E790E0DE
:1037F0000E94711240922005F0E3F09321058EE5BE
:103800000E94851B1092200520922105712C612CAD
:103810008981681648F580918D04F30196E0989FA0
:10382000E00DF11D1124EB52FE4F80810E94851B9B
:10383000EFEF6E1A7E0AECCF80E65812CDCF1093D0
:10384000750400937404F0927304E0927204D092B1
:103850007104C0927004E0E4F0E0F0938004E0931F
:103860007F0480E2582EB8CF409220052092210597
:10387000852D0E94851B0E94D4108111AFCF33206B
:1038800061F086E00E946E0E892B39F06AE070E0EC
:1038900080E090E00E947E0F312C86E00E946E0E48
:1038A000892B09F07DCF31107BCFA0908D04F6E0FD
:1038B000FA9D50011124C5018B529E4F5C01EA8193
:1038C000FB81E80FF91F50820E9411166AE070E038
:1038D00080E090E00E947E0FEA81FB813196FB83BD
:1038E000EA83F9E04F0E8DE248123ACFF5011582D6
:1038F0000F900F900F90DF91CF911F910F91FF903C
:10390000EF90DF90CF90BF90AF909F908F907F907F
:103910006F905F904F903F902F900895089590E0A2
:1039200080E00895FC0101900020E9F73197AF0194
:10393000481B590BBC0185EE94E00C94BC0F8F9290
:103940009F92AF92BF920F931F93CF93DF93CDB708
:10395000DEB7A1970FB6F894DEBF0FBECDBF19A298
:10396000423008F44AE08E010F5D1F4F842E912CE7
:10397000B12CA12CA50194010E94442AE62FB90183
:10398000CA01EA30F4F4E05DD801EE938D01232BF7
:10399000242B252B79F790E080E0109719F0CD01CA
:1039A0000E94921CA1960FB6F894DEBF0FBECDBF49
:1039B000DF91CF911F910F91BF90AF909F908F900B
:1039C0000895E95CE1CF4F925F926F927F928F9260
:1039D0009F92AF92BF92CF92DF92EF92FF920F939E
:1039E0001F93CF936B017C01742EAC019B010E944D
:1039F000B32C882399F081E292E0CF911F910F912F
:103A0000FF90EF90DF90CF90BF90AF909F908F90FE
:103A10007F906F905F904F900C94921C46015701DD
:103A2000E894B7F82FEF3FEF4FE75FE7C501B40128
:103A30000E94B32C81110DC02FEF3FEF4FE75FE7DE
:103A4000C501B4010E94E22A18161CF485E292E036
:103A5000D4CF2FEF3FEF4FE75FE4C701B6010E94DD
:103A6000412C18161CF489E292E0C7CF2FEF3FEFEC
:103A70004FE75FECC701B6010E94E22A87FDF3CF52
:103A800020E030E0A901C701B6010E94E22A10E05F
:103A900000E087FF08C08DE20E94851B8C01F7FAC9
:103AA000F094F7F8F094C0E060E070E080E09FE30D
:103AB0007C1641F020E030E040E251E40E94E72A29
:103AC000CF5FF6CFA70196010E94762A2B013C0119
:103AD0000E94602B4B015C014AE00E949F1C7C010C
:103AE000E00EF11ECC23B1F1C501B4010E948F2B71
:103AF0009B01AC01C301B2010E94752A4B015C011C
:103B00008EE20E94851BE80EF91EC15018F120E0DC
:103B100030E040E251E4C501B4010E94462C2B0183
:103B20003C010E94602B4B01B12CA12C4AE0C50145
:103B3000B4010E949F1CE80EF91EC501B4010E9449
:103B40008F2B9B01AC01C301B2010E94752A4B016E
:103B50005C01DBCFC701CF911F910F91FF90EF90D8
:103B6000DF90CF90BF90AF909F908F907F906F909D
:103B70005F904F9008957F928F929F92AF92BF92E5
:103B8000CF92DF92EF92FF920F931F93CF93DF9329
:103B90007C0186E00E946E0E11E0892B09F010E096
:103BA00091E4C92E9EE0D92E00E22AE0722EC09147
:103BB0007F04D0918004D595C7950E94A1104E0135
:103BC000B12CA12C8FE49EE00E94F80DD092FF044E
:103BD000C092FE04F7014081518160E080E00E94C4
:103BE000481210922005009321058FE192E00E9477
:103BF000921C7092200500932105209779F588E6A4
:103C000090E00E946A1B0E94D4108111DBCF112327
:103C100061F086E00E946E0E892B39F06AE070E058
:103C200080E090E00E947E0F10E086E00E946E0E21
:103C3000892B09F0BCCF1111BACF0E941116CE0109
:103C4000DF91CF911F910F91FF90EF90DF90CF9078
:103C5000BF90AF909F908F907F9008954AE0C501EC
:103C6000B4010E949F1C8DE292E00E94921CF70119
:103C700082819381009739F20E94921CC4CF1F93D6
:103C8000CF93DF93EC01162F0E94042A181739F006
:103C9000612FCE01DF91CF911F910C940C2ADF91FF
:103CA000CF911F910895AF92BF92CF92DF92EF9282
:103CB000FF920F931F93CF93DF9360918A0182E06D
:103CC00090E00E943F1E6091890183E090E00E9495
:103CD0003F1E6091840184E090E00E943F1E60914D
:103CE000830185E090E00E943F1E60917E0186E0A6
:103CF00090E00E943F1E6091D30187E090E00E9417
:103D00003F1E6091D20188E090E00E943F1E6091CA
:103D1000D10189E090E00E943F1E609190048AE00A
:103D200090E00E943F1E6091BE018BE090E00E94F7
:103D30003F1E6091B1018CE090E00E943F1E6091B7
:103D40008D048DE090E00E943F1E60916B018EE03B
:103D500090E00E943F1E8FE0E82EF12C10E006E07C
:103D600080916B011817B8F5109F60011124D0E005
:103D7000C0E0FE01EC0DFD1DEB52FE4F6081C7015E
:103D80008C0F9D1F0E943F1E2196C630D10589F7DA
:103D9000670186E0C80ED11C88E0189FE00111245D
:103DA000C55DDE4F8EE0E80EF11C69812296C601EA
:103DB0000E943F1E560182E0A80EB11CFE01329700
:103DC0006081C60101960E943F1E6501AE14BF04CA
:103DD00061F71F5FC5CFDF91CF911F910F91FF90CA
:103DE000EF90DF90CF90BF90AF9008950C94042A8D
:103DF0001F920F920FB60F9211242F933F938F9320
:103E00009F93AF93BF9380919F049091A004A09142
:103E1000A104B091A20430919E0423E0230F2D371A
:103E200058F50196A11DB11D20939E0480939F0417
:103E30009093A004A093A104B093A2048091A30442
:103E40009091A404A091A504B091A6040196A11D8F
:103E5000B11D8093A3049093A404A093A504B093F0
:103E6000A604BF91AF919F918F913F912F910F9099
:103E70000FBE0F901F90189526E8230F0296A11DE4
:103E8000B11DD2CF1F920F920FB60F9211242F9314
:103E90003F934F935F936F937F938F939F93EF9392
:103EA000FF9383B1817029B190916904981709F447
:103EB0009DC030E0220F232F221F330B922F8093BF
:103EC000690440916804241709F490C020936804A1
:103ED0002091700430917104981719F03195219553
:103EE000310940917F045091800460917404709175
:103EF0007504240F351F261737070CF48BC020914B
:103F0000700430917104981719F031952195310999
:103F100040917F0450918004609172047091730409
:103F2000240F351F621773070CF46FC040917004A3
:103F300050917104981719F05195419551092091AC
:103F40007F0430918004240F351F30938004209328
:103F50007F0441E0981340E020916704421709F480
:103F600040C02091700430917104981719F0319578
:103F70002195310960917F0470918004E09174046F
:103F8000F0917504260F371F2E173F070CF44CC015
:103F90002091700430917104981719F03195219592
:103FA000310960917F0470918004E0917204F09176
:103FB0007304260F371FE217F3078CF1209170046A
:103FC00030917104981719F031952195310980913C
:103FD0007F0490918004820F931F909380048093BC
:103FE0007F044093670481E080938C04FF91EF91FC
:103FF0009F918F917F916F915F914F913F912F9101
:104000000F900FBE0F901F90189520917204309161
:1040100073049BCF209174043091750496CF8091E6
:10402000720490917304D9CF8091740490917504B7
:10403000D4CF1895CF93DF93CDB7DEB72D970FB6BA
:10404000F894DEBF0FBECDBF789484B5826084BD86
:1040500084B5816084BD85B5826085BD85B581608C
:1040600085BD80916E00816080936E00109281000A
:1040700080918100826080938100809181008160C5
:104080008093810080918000816080938000809186
:10409000B10084608093B1008091B0008160809312
:1040A000B00080917A00846080937A0080917A00D9
:1040B000826080937A0080917A00816080937A0098
:1040C00080917A00806880937A001092C10060E04D
:1040D0008EE00E94C50E60E08FE00E94C50E61E098
:1040E00085E00E94C50E61E089E00E94C50E62E095
:1040F00087E00E94C50E62E088E00E94C50E62E083
:1041000086E00E94C50E62E08AE00E94C50E8FEF35
:1041100090E00E94010F60E085E00E94970E809180
:104120007A00876080937A0080917A00886080931B
:104130007A00789481E080936B00809368008BBB59
:104140008091F404883209F0B7C08FEF809309059D
:1041500090E080E00E94F61E182F81E090E00E941F
:10416000F61E912F8C36974E09F0B6C082E090E093
:104170000E94F61E182F83E090E00E94F61E912FF9
:1041800090938A018093890184E090E00E94F61E5A
:10419000182F85E090E00E94F61E912F90938401E5
:1041A0008093830186E090E00E94F61E80937E015A
:1041B00087E090E00E94F61E8093D30188E090E0B3
:1041C0000E94F61E8093D20189E090E00E94F61EC4
:1041D0008093D1018AE090E00E94F61E80939004C3
:1041E0008BE090E00E94F61E91E0811101C090E00A
:1041F0009093BE018CE090E00E94F61E91E0811148
:1042000001C090E09093B1018DE090E00E94F61E15
:1042100080938D048EE090E00E94F61E282E8093FD
:104220006B015BE2852E51E0952E65EDA62E61E0D7
:10423000B62E7FE0E72EF12C312C231409F458C060
:1042400010E000E0C701800F911F0E94F61EF501EB
:10425000E00FF11F80830F5F1F4F0630110591F7AC
:10426000670136E0C30ED11C27016EE0460E511CDB
:104270003401C6010E94F61E082F10E0102F0027FF
:10428000D3010D931C937601B2E0EB0EF11CC60135
:1042900001960E94F61E082BF301019311933F0132
:1042A00067014E145F0429F73394F8E08F0E911CD8
:1042B00026E0A20EB11CC1CF823011F483E046CFBC
:1042C000813009F443CF803309F042CF8FEF8093E0
:1042D000090580930A053CCF67EE90E080E00E94DC
:1042E0003F1E6CE681E090E00E943F1E0E94531E3C
:1042F0000E94531590936F0480936E040E94FB15E7
:1043000090938F0480938E040091890110918A010B
:1043100010938704009386048EE00E94CD15BC01A3
:1043200090E080E00E948F2B60936A0470936B048E
:1043300080936C0490936D040E948F150E94A819BD
:1043400020E030E040EA51E46091880470918904F3
:1043500080918A0490918B040E94762A6B017C01E3
:10436000B80190E080E00E948F2B9B01AC01C70157
:10437000B6010E94E22A87FF04C090E080E00E941C
:10438000010F1092DB041092DC041092DD041092F5
:10439000DE04412C512C3FE7632E33E4732E409210
:1043A000DF045092E0046092E1047092E204A09075
:1043B000C704B090C8048091E304D501CD90DD908E
:1043C000ED90FC90882309F4F6C6A3019201C70181
:1043D000B6010E94412C181634F5F5014082518235
:1043E000628273828090CF049090D004A090D10418
:1043F000B090D204C090DF04D090E004E090E104DB
:10440000F090E204A7019601C501B4010E94412C7D
:104410001816CCF4C092CF04D092D004E092D1040C
:10442000F092D20420C020E030E0A901C701B6011B
:104430000E94E22A87FFD6CFD5011D921D921D92C0
:104440001C921397CFCFC090DB04D090DC04E09097
:10445000DD04F090DE04A7019601C501B4010E94BD
:10446000E22A87FDD7CF81E08093E30483B1817096
:104470008093690489B190E0880F892F881F990B78
:1044800080936804209169049091680481E0291365
:1044900080E0809367048CE291E0909375048093B0
:1044A000740480E293E090937304809372048AE032
:1044B00090E09093710480937004000F111F10938B
:1044C000800400937F040E94B00F60938204709375
:1044D000830480938404909385040E9411160E94A3
:1044E0001116E0917F04F0918004FA87E987F59531
:1044F000E795FC87EB87F0938704E093860486E0DA
:104500000E946E0E8D8781116EC180917E0488237A
:1045100009F469C10E9411160E94B00F6B017C0161
:10452000C0927A04D0927B04E0927C04F0927D04E5
:1045300086E00E946E0E892B59F40E94B00F6C1910
:104540007D098E099F09643F71408105910580F3C3
:104550000E94B00F6C197D098E099F09643F71405C
:104560008105910508F4BAC58FEF90E00E94010F14
:104570000E94111610E0EAE02E2E312C412F62E14C
:104580008FEB91E00E948016182F873008F007C14A
:10459000E82FF0E0E253FD4D0C94C82CBD23C1265A
:1045A0003F27AC27BA27C427D22720E030E0A90153
:1045B000C701B6010E94E22A87FF55CF1092CF04AF
:1045C0001092D0041092D1041092D2044CCF8330B8
:1045D00009F46BC3843009F0E2C080916B0188302C
:1045E00008F0CCC391E0980F90936B0180938D04F9
:1045F0000E948A1BE0918D04B8E0EB9FF00111242A
:10460000E55DFE4F28ED30E03183208384E391E0C7
:1046100093838283A6E8B1E0B583A4838EE190E022
:1046200097838683AAC0B0908D0411E0B11001C0B9
:1046300010E080916B018150990B109275041092DB
:104640007404880F991F909373048093720481E01F
:1046500090E090937104809370048B2D90E0880F0C
:10466000991F9093800480937F0486E00E946E0ED1
:1046700001E0892B09F000E041E4442E4EE0542E85
:1046800056E0752EE0907F04F0908004F594E79456
:10469000AE2C6701DD24C601810F911D17FD9A958F
:1046A0008B19910910E097FD06C08330910514F035
:1046B00082E090E0182F0E94A110812F012E000CA3
:1046C000990B9C012F5F3F4FB22EB29420EFB22284
:1046D0006A2C611AC81AD90A8FE49EE00E94F80D6C
:1046E0005092FF044092FE0485EC90E00E9471120B
:1046F0004FE152E06B2D80E00E944812312C912C4A
:10470000812C862D830D339490916B01891780F451
:10471000C601880D991D789EA001799E500D112427
:104720004B525E4F632D6295607F8CE00E94481271
:104730003FEF831A930A63E03612E3CF0E94D4104E
:104740008111CACF002361F086E00E946E0E892B92
:1047500039F06AE070E080E090E00E947E0F00E0B7
:1047600086E00E946E0E892B09F06CC101116AC1AE
:104770000E941116A0928D0410E0412F6EE08CE68D
:1047800091E00E948016182F823009F48BC208F045
:104790001ECF882309F447CF813009F455C10E9408
:1047A000531E81E080938C04EB85FC85F093870495
:1047B000E09386048CE291E09093750480937404F6
:1047C00080E293E090937304809372048AE090E017
:1047D000909371048093700489859A858E7F90935D
:1047E000800480937F04FD85F0937E04809195047E
:1047F000882309F11091D1011123E9F00E94B00F33
:10480000C0907604D0907704E0907804F09079041A
:104810006C197D098E099F0928EE33E040E050E0D5
:104820000E94442A211738F0109295040E94111614
:1048300081E08093D40180918C048823E9F18091F8
:104840009604882349F120E030E040EA51E4609189
:1048500088047091890480918A0490918B040E944D
:10486000762A6B017C01609186047091870490E048
:1048700080E00E948F2B9B01AC01C701B6010E9412
:10488000E22A87FF04C090E080E00E94010F0E94AE
:10489000111681E08093D40110928C04109296043A
:1048A000109297040E94B00F609382047093830467
:1048B00080938404909385040E94B00F0091820439
:1048C000109183042091840430918504601B710B46
:1048D000820B930B20E63AEE40E050E00E94442A1F
:1048E000122F209381048091960481110BC0809136
:1048F000D301882339F0281728F081E080939604AB
:104900000E9411168091970481110BC08091D201F1
:10491000882339F0181728F081E0809397040E94CB
:1049200011160E94531A0E947B170E94A11001E4E5
:104930001EE088E2D82E93E5F92E2FE0C22E34E156
:10494000B32E44E3E42E56E0A52E65E2962E76E1E2
:10495000872E8FE49EE00E94F80D1093FF040093D1
:10496000FE044AE352E060E080E00E944812D092E8
:1049700020051092210560919A0470919B0480910A
:104980009C0490919D0440E00E94E31CF09220055D
:10499000109221058091980490919904853F91404F
:1049A00008F4B2C382E691E00E946A1B80919004F1
:1049B000882309F4DBC360918E0470918F0490E02A
:1049C00080E00E948F2B20E030E04AE754E40E9410
:1049D000E72A2B013C0110922005E09221058091ED
:1049E0008D048A9DC00111248B529E4F0E94921CFF
:1049F000F0922005E092210541E0C301B2010E943E
:104A0000E31C8CE391E00E946A1B80EA9AE00E941A
:104A1000F80D1093FF040093FE04909220058092FD
:104A20002105609198047091990488E391E0653FB5
:104A300031E0730708F0B1C390E080E04AE00E94E3
:104A40009F1CADC3BE2C1ECECE0101963C01C12CD5
:104A5000D12C7601C39488EC282E312C91E4492E78
:104A60009EE0592EE0918D0494E0E99FF00111241D
:104A7000C6010197E80FF91FEE0FFF1FE55DFE4F1E
:104A8000808191819093870480938604309275048D
:104A900020927404A8EEB3E0B0937304A093720460
:104AA000E1E0F0E0F0937104E0937004880F991F47
:104AB0009093800480937F04F1E0F093D40186E02A
:104AC0000E946E0E01E0892B09F000E00E94531A4B
:104AD0000E947B170E94A1108FE49EE00E94F80DB7
:104AE0005092FF044092FE0481E091E00E94711216
:104AF0001092200520E1209321058AEF90E00E948A
:104B00006A1B4AE0C701B6010E949F1C8FE292E037
:104B10000E94921C8091050210922005882309F4BE
:104B2000A1C030E2309321058DEE90E00E946A1B17
:104B30001092200560E36093210586EE90E00E94CC
:104B40006A1B80917F0490918004959587954C0114
:104B5000092E000CAA08BB0897FF80C08DE20E94B6
:104B6000851B66277727CB01681979098A099B0974
:104B70004AE00E949F1C0E94D4108111ADCF0023F7
:104B800061F086E00E946E0E892B39F06AE070E0D9
:104B900080E090E00E947E0F00E086E00E946E0EB2
:104BA000892B09F093CF011191CF80917F049091CF
:104BB000800495958795D3018D939D933D010E9427
:104BC00011166AE070E080E090E00E947E0FBFEF77
:104BD000CB1ADB0AEB0AFB0AE4E0CE16D104E104AF
:104BE000F10409F03FCF8FEF90E00E94010F8BEAB4
:104BF00094E00197F1F70E948F150E94602B2B0122
:104C000078876F83A980BA80EB80FC80C5010A9603
:104C10008E159F0508F0B1CDCD80DE80C7010A96C4
:104C20008C159D0508F0A9CD40E066E08FE091E08D
:104C30000E948016882309F4A0CDE0918D0428E01D
:104C4000E29FF0011124E55DFE4FB182A082F38264
:104C5000E282D582C482578246828FCD4AE0C50166
:104C6000B40187CF80E2809321058FED90E00E9410
:104C70006A1B60916A0470916B0480916C0490913E
:104C80006D040E94602B90E080E04AE00E949F1C2F
:104C90001092200590E39093210580ED90E00E9412
:104CA0006A1B69CF0E948A1B68CD80916B0181309D
:104CB00029F485E191E00E942F165FCD40E066E087
:104CC0008DE191E00E948016882309F456CD8091F1
:104CD0008D0490916B01A92FA150BB0BAD0106E093
:104CE0008A171B0639F4815080938D04915090935C
:104CF0006B0143CDE82FF0E0E417F507BCF7809F88
:104D00007001112430E020E05F01BFEFAB1ABB0A55
:104D1000B9016E0D7F1D6B527E4FDB011696DC9044
:104D20001697DC922F5F3F4F2630310589F7D5016A
:104D300023E0AA0FBB1F2A95E1F7A55DBE4F2D9179
:104D40003C91119763E0EE0FFF1F6A95E1F7E55D77
:104D5000FE4F3183208312962D913C91139733831C
:104D6000228314962D913C911597358324831696B2
:104D70002D913C91378326838F5FBCCF83E291E0F6
:104D80009ACF00E048E2442E512C50E9652E77245A
:104D900073946CE2862E9924939470E2A72E73E0AC
:104DA000B72EE4E1CE2ED12CF8ECEF2EF12C402FD3
:104DB0006AE08BE891E00E948016082F813009F4A8
:104DC0003FC0F8F0823009F0D9CB80917E0190E0AD
:104DD000D0927504C0927404F0927304E09272044D
:104DE0003092710420927004880F991F9093800470
:104DF00080937F048AE791E00E94BB1D80937E012F
:104E0000D6CF8091890190918A0190927504809209
:104E10007404B0927304A0927204309271042092D0
:104E20007004880F991F9093800480937F0485E815
:104E300091E00E94BB1D90938A0180938901B7CFB6
:104E40008091830190918401509275044092740482
:104E50007092730460927204309271042092700414
:104E6000880F991F9093800480937F048FE791E0CF
:104E70000E94BB1D909384018093830198CF00E032
:104E8000402F6AE081EA91E00E948016082F81306D
:104E900009F442C008F1823009F070CB8091D10151
:104EA00090E0109275041092740428E631E030937B
:104EB0007304209372043092710420927004880F5E
:104EC000991F9093800480937F0485E991E00E946C
:104ED000BB1D8093D101D4CF8091D30190E010927B
:104EE000750410927404ECE3F0E0F0937304E09323
:104EF000720421E030E03093710420937004880F35
:104F0000991F9093800480937F048DE991E00E9423
:104F1000BB1D8093D301B4CF8091D20190E0109259
:104F2000750410927404A8E7B0E0B0937304A093E2
:104F30007204E5E0F0E0F0937104E0937004880FF0
:104F4000991F9093800480937F0489E991E00E94E7
:104F5000BB1D8093D20194CF4091BE0166E088EBE7
:104F600091E00E94801691E0811101C090E0909341
:104F7000BE0104CB4091900466E082EB91E00E9478
:104F8000801680939004FACA4091B10166E08BEAE2
:104F900091E00E94801691E0811101C090E0909311
:104FA000B101ECCA86E00E946E0E01E0892B09F087
:104FB00000E00E94531590936F0480936E04BC012F
:104FC00090E080E00E948F2B20E030E04AE754E43C
:104FD0000E94E72A6B017C010E94FB1590938F04CD
:104FE00080938E04BC0190E080E00E948F2B20E033
:104FF00030E04AE754E40E94E72A4B015C010E943A
:105000008F152B013C010E94A1108FE49EE00E94AD
:10501000F80D81E49EE09093FF048093FE041092CB
:1050200020051092210589E291E00E946A1B85E328
:1050300092E00E94921C1092200590E1909321052D
:1050400083E291E00E946A1B41E0C301B2010E9429
:10505000E31C80E291E00E946A1B10922005A0E20E
:10506000A09321058AE191E00E946A1B41E0C501FD
:10507000B4010E94E31C87E191E00E946A1B109238
:105080002005B0E3B093210580E191E00E946A1B06
:1050900041E0C701B6010E94E31C8DE091E00E944F
:1050A0006A1B0E94D4108111B0CF002361F086E00A
:1050B0000E946E0E892B39F06AE070E080E090E08B
:1050C0000E947E0F00E086E00E946E0E892B09F0A0
:1050D00070CF01116ECF0E94111650CA80919504B5
:1050E00091E0892780939504882351F00E94B00FA6
:1050F0006093760470937704809378049093790496
:1051000081E080938C046FCB80919704882319F001
:105110008CE591E049CC80919604882319F086E5CE
:1051200091E042CC80919504882319F080E591E0CC
:105130003BCC80910502882319F08AE491E034CCBD
:1051400020E030E044E353E46091910470919204D4
:1051500080919304909194040E94E22A87FF03C0F7
:1051600084E491E021CC8EE391E01ECC82EC91E0CE
:105170000E94F80D1093FF040093FE04C0922005D6
:10518000B09221056091980470919904653F81E087
:10519000780708F451CC84E391E00E946A1B0E94D6
:1051A000D4108111D6CB80E090E0892B09F499C905
:1051B0000E94000096C9C092CF04D092D004E09221
:1051C000D104F092D204E091C504F091C60480812C
:1051D0009181A281B3818093D3049093D404A0934E
:1051E000D504B093D60420E030E04FE753E4C70184
:1051F000B6010E94412C18160CF0D7C94092CF047A
:105200005092D0046092D1047092D2042CC90F93B2
:105210001F93CF9381E994E09093C8048093C704CF
:1052200083E694E09093C6048093C5048AE994E0F1
:105230009093CA048093C9041092E3041092DB0493
:105240001092DC041092DD041092DE0480E090E005
:10525000AFE7B3E48093DF049093E004A093E1040C
:10526000B093E20484E690E0A0E0B0E08093D7043D
:105270009093D804A093D904B093DA0481E090E02D
:105280009093C2048093C1049093C4048093C30498
:10529000C1E0C093E40480E090E0A0E3B1E4809337
:1052A000A9049093AA04A093AB04B093AC0480E04B
:1052B00090E0A0E0BFE38093AD049093AE04A09390
:1052C000AF04B093B00480E090E0A0E8BFE3809327
:1052D000B1049093B204A093B304B093B40480E0FB
:1052E00090E0A0E3B1EC8093B5049093B604A09352
:1052F000B704B093B8048DEC9CECACE4BDEB8093A8
:10530000B9049093BA04A093BB04B093BC0480E0AA
:1053100090E0A0E2B1EC8093BD049093BE04A09312
:10532000BF04B093C0040E94B00F0091D704109145
:10533000D8042091D9043091DA04601B710B820BE0
:10534000930B6093CB047093CC048093CD04909323
:10535000CE041092E8041092E7048AE092E0909361
:10536000E6048093E5041092200510922105109226
:1053700022051092EE041092ED041092F0041092A7
:10538000EF041092F204C093F10482E28093F304DC
:105390001092F8041092F704ECE0F5E08AE195E051
:1053A0002FEF21938E179F07E1F781E08093090586
:1053B00026EF3DE03093FF042093FE048093000528
:1053C000109201051092020580E48093030510926B
:1053D000040589EE9FE090931B0580931A0589E0F0
:1053E00091E09093EC048093EB0482E180931705A5
:1053F0000E943B108AE092E09093E6048093E504DB
:10540000CF911F910F910895F999FECF92BD81BD63
:10541000F89A992780B50895262FF999FECF1FBADB
:1054200092BD81BD20BD0FB6F894FA9AF99A0FBECD
:1054300001960895052E97FB1EF400940E94312AD0
:1054400057FD07D00E94442A07FC03D04EF40C9469
:10545000312A50954095309521953F4F4F4F5F4FE2
:10546000089590958095709561957F4F8F4F9F4FD0
:1054700008950E94662AA59F900DB49F900DA49F49
:10548000800D911D11240895A1E21A2EAA1BBB1BA9
:10549000FD010DC0AA1FBB1FEE1FFF1FA217B30700
:1054A000E407F50720F0A21BB30BE40BF50B661F16
:1054B000771F881F991F1A9469F7609570958095DA
:1054C00090959B01AC01BD01CF010895A29FB00151
:1054D000B39FC001A39F700D811D1124911DB29F28
:1054E000700D811D1124911D08955058BB27AA27C6
:1054F0000E948D2A0C94072C0E94F92B38F00E94F0
:10550000002C20F039F49F3F19F426F40C94F62B6C
:105510000EF4E095E7FB0C94F02BE92F0E94182C79
:1055200058F3BA17620773078407950720F079F4D8
:10553000A6F50C943A2C0EF4E0950B2EBA2FA02D64
:105540000B01B90190010C01CA01A0011124FF2730
:10555000591B99F0593F50F4503E68F11A16F0402B
:10556000A22F232F342F4427585FF3CF469537952A
:105570002795A795F0405395C9F77EF41F16BA0BEF
:10558000620B730B840BBAF09150A1F0FF0FBB1F9D
:10559000661F771F881FC2F70EC0BA0F621F731FE6
:1055A000841F48F4879577956795B795F7959E3F43
:1055B00008F0B0CF9395880F08F09927EE0F9795D4
:1055C000879508950E94CC2B08F481E008950E94ED
:1055D000FB2A0C94072C0E94002C58F00E94F92BF7
:1055E00040F029F45F3F29F00C94F02B51110C94FA
:1055F0003B2C0C94F62B0E94182C68F39923B1F3E2
:10560000552391F3951B550BBB27AA2762177307E8
:10561000840738F09F5F5F4F220F331F441FAA1F7C
:10562000A9F335D00E2E3AF0E0E832D09150504038
:10563000E695001CCAF72BD0FE2F29D0660F771FE6
:10564000881FBB1F261737074807AB07B0E809F0CC
:10565000BB0B802DBF01FF2793585F4F3AF09E3F51
:10566000510578F00C94F02B0C943B2C5F3FE4F345
:10567000983ED4F3869577956795B795F7959F5F94
:10568000C9F7880F911D9695879597F90895E1E0E0
:10569000660F771F881FBB1F621773078407BA073F
:1056A00020F0621B730B840BBA0BEE1F88F7E0959A
:1056B00008950E94602B6894B1110C943B2C0895BE
:1056C0000E94202C88F09F5798F0B92F9927B75146
:1056D000B0F0E1F0660F771F881F991F1AF0BA9596
:1056E000C9F714C0B13091F00E943A2CB1E008958E
:1056F0000C943A2C672F782F8827B85F39F0B93F80
:10570000CCF3869577956795B395D9F73EF4909548
:105710008095709561957F4F8F4F9F4F0895E894C6
:1057200009C097FB3EF490958095709561957F4FE9
:105730008F4F9F4F9923A9F0F92F96E9BB27939597
:10574000F695879577956795B795F111F8CFFAF4A7
:10575000BB0F11F460FF1BC06F5F7F4F8F4F9F4FD8
:1057600016C0882311F096E911C0772321F09EE836
:10577000872F762F05C0662371F096E8862F70E09C
:1057800060E02AF09A95660F771F881FDAF7880F76
:105790009695879597F90895990F0008550FAA0BCC
:1057A000E0E8FEEF16161706E807F907C0F0121634
:1057B0001306E407F50798F0621B730B840B950B37
:1057C00039F40A2661F0232B242B252B21F408958C
:1057D0000A2609F4A140A6958FEF811D811D089529
:1057E00097F99F6780E870E060E008959FEF80EC94
:1057F000089500240A941616170618060906089537
:1058000000240A9412161306140605060895092E9C
:105810000394000C11F4882352F0BB0F40F4BF2B0B
:1058200011F460FF04C06F5F7F4F8F4F9F4F08954B
:1058300057FD9058440F551F59F05F3F71F0479541
:10584000880F97FB991F61F09F3F79F08795089526
:10585000121613061406551FF2CF4695F1DF08C045
:10586000161617061806991FF1CF86957105610562
:1058700008940895E894BB2766277727CB0197F90A
:1058800008950E94CC2B08F48FEF08950E94592CA4
:105890000C94072C0E94F92B38F00E94002C20F069
:1058A000952311F00C94F02B0C94F62B11240C94EE
:1058B0003B2C0E94182C70F3959FC1F3950F50E07C
:1058C000551F629FF001729FBB27F00DB11D639FB2
:1058D000AA27F00DB11DAA1F649F6627B00DA11D58
:1058E000661F829F2227B00DA11D621F739FB00DFE
:1058F000A11D621F839FA00D611D221F749F33276E
:10590000A00D611D231F849F600D211D822F762F06
:105910006A2F11249F5750409AF0F1F088234AF0E3
:10592000EE0FFF1FBB1F661F771F881F915050404F
:10593000A9F79E3F510580F00C94F02B0C943B2C62
:105940005F3FE4F3983ED4F3869577956795B795D6
:10595000F795E7959F5FC1F7FE2B880F911D9695F0
:10596000879597F908950E94CC2B880B990B089581
:10597000DB018F939F930E94392ABF91AF91A29F21
:10598000800D911DA39F900DB29F900D112408953D
:10599000EE0FFF1F0590F491E02D0994F894FFCFCE
:1059A000084000000080E203FF281400014A133F72
:1059B000025002530257025F026A027602800250CE
:1059C00002530257028F029B02AA02D800340186BA
:1059D000011E0000000000000000000000000000A8
:1059E00000000000000000000000000000000000B7
:1059F00000000000000000000000000000000000A7
:105A00000000000000000000000000011A02B302C4
:105A1000BE02CC02D702E202EE02F5020003320619
:105A200003000396001103000340011E0311030647
:105A300003F502EE022C03380340034A0352034AE3
:105A4000035E03520340032C03EE026D0374037CD8
:105A5000030183038F039B03A603B303BA0301BEB1
:105A600003C9031E035E03A60383036D03D603EE7F
:105A700002280F05014243312E35000000000000CE
:105A80000000000000000000000000000000000016
:105A90000000000000000000000000000000000006
:105AA00000000000000100000000431BBC0F8F1C21
:105AB0008E1C000100FF0100FF005469703A003E97
:105AC000006E616E00696E66006F766600200020D1
:105AD0006F6620330076312E34005345543A00531C
:105AE000746F72652053657474696E6773203F002C
:105AF0004E6F00596573005761726E696E67005989
:105B00006F752063616E6E6F740064656C6574659B
:105B100020796F7572006C61737420746970210054
:105B200041726520796F752073757265203F005949
:105B30006F752072656163686564006D6178696D79
:105B4000756D206E756D626572006F662074697088
:105B50007321004368616E6765205469700043617A
:105B60006C696272617465205469700052656E617F
:105B70006D65205469700044656C657465205469D6
:105B80007000416464206E6577205469700052652E
:105B90007475726E00426F6F73742054656D70007F
:105BA000646567204300536C6565702054656D70B3
:105BB0000044656661756C742054656D70005465B1
:105BC0006D702053657474696E677300426F6F73F4
:105BD000742054696D6572005365636F6E64730061
:105BE0004F66662054696D6572004D696E75746507
:105BF0007300536C6565702054696D65720054695B
:105C00006D65722053657474696E67730042757AAE
:105C10007A65720044697361626C6500456E616209
:105C20006C65004D61696E2053637265656E00425C
:105C30006967204E756D62657273004D6F726520E5
:105C4000496E666F7300436F6E74726F6C20547987
:105C5000706500446972656374005049440053657F
:105C6000747570204D656E750054697020536574AD
:105C700074696E677300496E666F726D6174696FE7
:025C80006E00B4
:00000001FF
